:100000000C9411060C948F280C94BC280C9439067F
:100010000C9439060C9439060C9439060C94390664
:100020000C9439060C9439060C94840C0C94390603
:100030000C9439060C9439060C9439060C94390644
:100040000C94E9280C9439060C94812C0C94BC2C4B
:100050000C9439060C9439060C9439060C94390624
:100060000C9439060C943906EC1BF31BF31BEC1BA8
:10007000F31BF31BF31BF31BF31BF31BF31BF31B10
:10008000F31BF31BF31BF31BF31B611BF31BF31B92
:10009000F31BF31BF31BC41AF31BF31BF31BF31B20
:1000A000F31BF31BF31BF31BF31BF31BF31BF31BE0
:1000B000F31BF31BF31B6D1B6D1B6D1B6D1B6D1B6E
:1000C0006D1B6D1B6D1B6D1BF31BF31BF31BF31BD8
:1000D000F31BF31BC91A6C1B6C1B6C1B6C1BF31BF7
:1000E0007D1B851B8D1B951B9D1BA51BAD1BB51B70
:1000F000BF1BC91BD31BDD1B101BD01AF31BF31B2B
:10010000F31BF31B611BF31BF31BF31BF31BF31B11
:10011000F31BF31BF31B6B1B6B1B6B1B6B1BF31B8F
:100120007D1B851B8D1B951B9D1BA51BAD1BB51B2F
:10013000BF1BC91BD31BDD1B101BD01AF31BF31BEA
:10014000F31BF31B611B241C241C241C241C241CD7
:10015000241C241C241C241C241C241C241C241C9F
:10016000441D441D441D441D441D441D6B1C751C31
:100170007F1C891CEF1CF91C071D181DB51D251EB1
:10018000F61DFB1D001E051E0A1E0F1E141E251E39
:100190001F1E1E2533253F25482555257B258325F4
:1001A000A6259325456E746572206D656E752E2E9D
:1001B0002E00546F67676C6564206D6963726F50C1
:1001C000504D00546F67676C656420696E76657288
:1001D0007465642050504D2100546F67676C6564EE
:1001E000205458206D7574696E672100546F6767DD
:1001F0006C65642074656C656D657472792100505E
:10020000726F746F636F6C206572726F72207769A2
:1002100074682052580054696D656F757420776852
:10022000656E20636F6E6E656374696E6720746FB0
:1002300020525800507265737320616E79206B658F
:100240007920746F2063616E63656C00436F6E6E1E
:10025000656374696E6720746F2052582C20706F2C
:100260007765722075702074686520525820287751
:100270006974682062696E6420706C7567206966B5
:10028000206E6F74207573696E6720616C77617979
:10029000732062696E642900546F67676C6564201F
:1002A00027696D6D656469617465206F757470751B
:1002B000742700546F67676C65642027736C6176E0
:1002C00065206D6F64652700546F67676C656420F7
:1002D00027616C776179732062696E642700546FBF
:1002E00067676C65642050504D206368616E6E6571
:1002F0006C206C696D6974005365742052535349C6
:1003000020696E6A656374696F6E206368616E6EE2
:10031000656C2028303D3D64697361626C6529001D
:100320005365742050504D206D696E696D756D2058
:1003300073796E630053657420626561636F6E202C
:10034000696E74657276616C0053657420626561D4
:10035000636F6E2064656C6179005365742062651B
:1003600061636F6E206672657175656E6379206971
:100370006E20487A3A20303D64697361626C652C66
:100380002050783D504D52206368616E6E656C2040
:10039000782C2046783D465253206368616E6E6526
:1003A0006C2078005365742050574D2073746F7023
:1003B0002064656C61792028302064697361626C07
:1003C00065642C20312D323535203D3D20302E31D5
:1003D00073202D2035306D696E29005365742050CF
:1003E000504D2073746F702064656C6179202830E3
:1003F0002064697361626C65642C20312D3235355F
:10040000203D3D20302E3173202D2035306D696E1A
:100410002900536574206661696C736166652064A8
:10042000656C61792028302064697361626C656451
:100430002C20312D323535203D3D20302E3173209A
:100440002D2035306D696E29002A2A2A2A2A2A2A67
:100450002A2A2A2A2A2A2A2A2A2A2A2A2A2A2A2AFC
:100460002A2A2A2A2A2A0052582041636B656420CE
:100470002D2072657665727420737563636573737E
:1004800066756C21002A2A2A2A2A2A2A2A2A2A2A36
:100490002A2A2A2A2A2A2A2A2A2A2A2A2A2A2A2ABC
:1004A0002A2A002A2A2A2A2A2A2A2A2A2A2A2A2AD6
:1004B0002A2A2A2A2A2A2A2A2A2A2A2A2A2A2A2A9C
:1004C0000052582041636B6564202D207570646173
:1004D0007465207375636365737366756C21002A98
:1004E0002A2A2A2A2A2A2A2A2A2A2A2A2A2A2A2A6C
:1004F0002A2A2A2A2A2A2A2A2A2A2A2A0056616CE1
:1005000069642063686F69636573206172653A206E
:100510005B315D2D5B31365D20286368616E6E65F1
:100520006C20312D31362900536574206F7574703D
:10053000757420666F7220706F727420005B585D56
:100540002061626F7274206368616E6765732061F9
:100550006E64206578697420525820636F6E6669F6
:1005600067005B535D207361766520736574746901
:100570006E677320746F205258005B525D20726565
:10058000766572742052582073657474696E67734F
:1005900020746F2064656661756C747300557365B3
:1005A000206E756D62657273205B312D445D207421
:1005B0006F206564697420706F727473205B452DC1
:1005C000515D20666F722073657474696E67730085
:1005D000202D20726563656976657220636F6E6693
:1005E0006967757261746F722C207278207377203E
:1005F000000A0A6F70656E4C52536E672000536597
:10060000742073657269616C2062617564726174D3
:10061000653A200056616C69642063686F696365A0
:10062000733A2031202D20342B34202F2032202DDE
:100630002038202F2033202D20382B34202F203419
:10064000202D203132202F2035202D2031322B3407
:10065000202F2036202D203136005365742043682A
:10066000616E6E656C20636F6E6669673A20005339
:1006700065742044617461726174652028302D3284
:10068000293A200053657420486F70206368616EBA
:100690006E656C7320286D61782032342C20736570
:1006A0007061726174656420627920636F6D6D6141
:1006B00073292076616C69642076616C756573209E
:1006C000312D3235353A2000536574206368616EF0
:1006D0006E656C2073706163696E672028783130B5
:1006E0006B487A293A200053657420524620706F77
:1006F0007765722028302D37293A20005365742001
:100700005246206D616769632028686578292065F5
:100710002E672E20307844454144463030443A20FC
:10072000005365742062617365206672657175653A
:100730006E63792028696E20487A293A20005B5A36
:100740005D20656E74657220726563656976657299
:1007500020636F6E66696775726174696F6E20756C
:1007600074696C79005B465D20646973706C6179B3
:100770002061637475616C206672657175656E6366
:100780006965732075736564005B525D2063616CFD
:1007900063756C6174652072616E646F6D206B654A
:1007A0007920616E6420686F70206C697374005BDF
:1007B000495D207265696E697469616C697A65204A
:1007C00073657474696E677320746F20736B6574DE
:1007D00063682064656661756C7473005B585D20A6
:1007E000726576657274206368616E6765732061F7
:1007F0006E642065786974206D656E75005B535D6D
:1008000020736176652073657474696E67732074F4
:100810006F20454550524F4D20616E6420657869C8
:1008200074206D656E7500557365206E756D62651B
:100830007273205B302D395D20746F20656469749C
:1008400020706172616D657465727300202D205394
:10085000797374656D20636F6E6669677572617414
:10086000696F6E000A0A6F70656E4C52536E672096
:10087000005129204F7574707574206265666F721F
:1008800065206C696E6B20283D465329203A200074
:10089000502920536C617665206D6F646520286552
:1008A00078706572696D656E74616C293A20004FCD
:1008B000292054696D65642042494E4420617420AA
:1008C0007374617274757020203A20004E29205094
:1008D000504D206F7574707574206C696D69746506
:1008E0006420202020203A200044495341424C45B6
:1008F00044004D292050504D205253534920746FCD
:10090000206368616E6E656C202020203A20004CC8
:10091000292050504D206D696E696D756D20737979
:100920006E63202875732920203A200044495341E2
:10093000424C4544004B29204661696C73616665F1
:1009400020626561636F6E20696E74762E20283197
:100950002D32353573293A20004A29204661696CC9
:100960007361666520626561636F6E2064656C61AA
:10097000792028302D323535203D3E20313073200E
:100980002D203135306D696E293A200049292046E5
:1009900061696C7361666520626561636F6E206674
:1009A00072712E203A200048292050574D20737430
:1009B0006F702064656C6179202020202020203A0F
:1009C000200047292050504D2073746F70206465BB
:1009D0006C6179202020202020203A200046292008
:1009E0004661696C736166652064656C617920207D
:1009F00020202020203A200050574D206368616E4F
:100A00006E656C200066756E6374696F6E3A2000C7
:100A10002920706F727420004454462055484620A7
:100A200033322D6269742031306368004F70656E17
:100A30004C52536E675258206D696E6920342F36C0
:100A4000636800466C7974726F6E2F4F72616E67C7
:100A50006552582055484620386368005258207423
:100A60007970653A200044697361626C656400487E
:100A70007A00203D3D200043616C63756C617465B4
:100A800064207061636B657420696E746572766151
:100A90006C3A20004229204D6963726F20286861FA
:100AA0006C66292050504D202020203A00412920FA
:100AB000496E7665727465642050504D20696E20D1
:100AC000202020203A003029204D75746520627561
:100AD0007A7A657220286D6F73746C79293A0039BF
:100AE000292053657269616C20626175647261745A
:100AF000653A00736D617274506F72740046725380
:100B00006B79005472616E73706172656E7400442B
:100B1000697361626C65640038292054656C656D89
:100B2000657472793A202020202020200037292067
:100B30004368616E6E656C20636F6E6669673A200C
:100B40002000362920446174617261746520283068
:100B50002D32293A20202000352920486F7020634B
:100B600068616E6E656C733A202020202000342965
:100B7000204368616E6E656C2073706163696E6797
:100B80003A202000332920524620706F776572206A
:100B900028302D37293A20202000322920524620A3
:100BA0006D616769633A20202020202020202000EA
:100BB00031292042617365206672657175656E63C7
:100BC000793A2020200000000000240027002A009D
:100BD00000000000250028002B000000000023007A
:100BE000260029000404040404040404020202028E
:100BF00002020303030303030102040810204080E0
:100C0000010204081020010204081020000000075F
:100C100000020100000304060000000000000000C4
:100C2000642E11241FBECFEFD8E0DEBFCDBF13E08E
:100C3000A0E0B1E0EAE0FFE502C005900D92A63920
:100C4000B107D9F716E0A6E9B3E001C01D92A934B7
:100C5000B107E1F71CE0C2E2DCE004C02297FE012C
:100C60000E94602FC032D107C9F70E94A92E0C94B0
:100C7000832F0C940000A0E0B0E0E1E4F6E00C94D7
:100C80002F2FEC01A880B980CA80DB80A114B104A9
:100C9000C104D10441F484E2A82E89EDB82E8BE57D
:100CA000C82E87E0D82EC601B5012DE133EF41E013
:100CB00050E00E940C2F27EA31E440E050E00E940F
:100CC000B82E7B018C01C601B5012DE133EF41E067
:100CD00050E00E940C2FCA01B9012CEE34EF4FEF07
:100CE0005FEF0E94B82E6E0D7F1D801F911F97FF32
:100CF00004C06150704080409048688379838A8343
:100D00009B839B01AC015F77B901CA01CDB7DEB708
:100D1000EAE00C944B2F0E943B06089581EB92E091
:100D20000E943B0608956093B1027093B2028093D3
:100D3000B3029093B4020895A0E0B0E0E2EAF6E0D6
:100D40000C94282FEC012B016A016115710519F033
:100D5000FB0191838083C114D10449F0C60102973D
:100D6000839728F020E030E040E050E0DCC0A9901C
:100D70008A2D90E00E94782F892BC9F7FDE2AF16EB
:100D800021F4A9903324339405C08BE2A81609F40A
:100D9000A9903324C114D10421F0E0E1CE16D1048E
:100DA00011F5F0E3AF1669F48881883711F08835C2
:100DB00041F4A980229682E0382A20E1C22ED12C6B
:100DC00012C0C114D10479F4E0E3AE1659F199E9E7
:100DD000E92E99E9F92E99E9092F99E1192F8AE06D
:100DE000C82ED12C3AC0FAE0CF16D10491F080E1A0
:100DF000C816D10429F0E8E0CE16D104F9F415C0E4
:100E0000BFEFEB2EBFEFFB2EBFEF0B2FBFE01B2F73
:100E100024C0A9E9EA2EA9E9FA2EA9E90A2FA9E135
:100E20001A2F1BC0F8E0CF2ED12CEFEFEE2EEFEFF4
:100E3000FE2EEFEF0E2FEFE11E2F0FC0960144277D
:100E400037FD4095542F6FEF7FEF8FEF9FEF0E949C
:100E5000EA2EC901DA017C018D0120E030E040E09A
:100E600050E060E03601882477FC8094982C70ED87
:100E7000B72EBA0CF9E0FB1570F48A2D81548A3133
:100E800018F499ECB92E06C08A2D81568A3148F59E
:100E900089EAB82EBA0C8B2D90E08C159D050CF5C7
:100EA0006F3FE9F0E216F30604071507B8F0CA0130
:100EB000B901A40193010E94B82E9B01AC018B2DB6
:100EC00090E0A0E0B0E0280F391F4A1F5B1F2817F1
:100ED00039074A075B0710F061E001C06FEFA99086
:100EE000C6CF4114510451F0662311F0219703C07D
:100EF00031FE04C02297F201D183C08330FE07C0C7
:100F000050954095309521953F4F4F4F5F4F67FF6C
:100F10000AC082E290E090934806809347062FEF44
:100F20003FEF4FEF5FEFB901CA01CDB7DEB7E1E1A7
:100F30000C94442FFC0188279927E89421912032B2
:100F4000E9F3293010F02E30C8F32B3241F02D3266
:100F500039F4689404C00E94EF07820F911D21911B
:100F600020532A30C0F31EF4909581959F4F089529
:100F700046E953E00E94BD070895009731F4DA0175
:100F80008D919C91009709F40EC0DC01FB013D910D
:100F90002191222319F03217C9F3FACF332331F408
:100FA000DA011D921C928827992708951197AF9313
:100FB000BF93FB013D912191321771F4332321F44A
:100FC00088279927119702C01E921196FA01A193C2
:100FD000B0839F918F910895222369F7EACF7AE039
:100FE000979F902D879F802D910D112408958091BA
:100FF0009803813019F482E08093980380919803DC
:10100000833019F484E0809398030895E3E0F0E0DE
:1010100089E080935700849190E08670863009F4CF
:1010200091E0892F08951F93182F0E9406088823A6
:1010300079F09FB781E080938F05F894A89588E1B7
:101040008093600010936000112309F0A8959FBF62
:101050001F910895382F20E080912105909122055D
:101060008227932740E061E270E19C01220F331F49
:1010700097FF04C0C9018627972701C0C9014F5FA8
:10108000483099F79093220580932105089586E3CF
:101090008093BE0380E092ECA1E0B0E08093BF03B8
:1010A0009093C003A093C103B093C20387E08093E1
:1010B000CB0380EC92E9ADEEB9E18093C30390934A
:1010C000C403A093C503B093C60385E08093CC030B
:1010D0008DEE9EEFADEABEED8093C7039093C803FB
:1010E000A093C903B093CA03ADECB3E080E090E0F5
:1010F000863010F0E0E004C0FC01E058FC4FE081D5
:10110000ED9301968831910599F782E08093E5038C
:101110008AE08093E603089580EC91EDA8E9BBE1B5
:1011200080939B0390939C03A0939D03B0939E0395
:1011300010929F031092A0031092A1031092A20399
:1011400008958436910520F4BC0180E090E025C02C
:101150008E3B910550F48A559040BC0180E090E0B0
:101160002AE030E040E050E016C0823D910550F4A6
:10117000845B9040BC0180E090E024E630E040E0F9
:1011800050E009C08D5C9040BC0180E090E028E513
:1011900032E040E050E00E94B82E24E630E040E02B
:1011A00050E00E94B82E089590E08C599F4F0E9405
:1011B000A1080895DC019896EC91F0E0E770F070DA
:1011C000E858FC4F808108958F929F92AF92BF9212
:1011D000CF92DF92EF92FF920F931F938C010E94A8
:1011E000DA08D80197962C9130E043E150E0249F33
:1011F000F001259FF00D349FF00D1124EB54FD4FAD
:1012000080809180A280B38090E00F96AA2797FDFE
:10121000A095BA2FBC01CD0120E43FE14DE750E09D
:101220000E94B82EA50194010E94EA2E69017A015C
:1012300080ED97E0A0E0B0E0C80ED91EEA1EFB1ECC
:10124000D80198968C91887181F060E07EEE8AEBEF
:101250009BE0A50194010E94EA2E28513C4F4F4F7C
:101260005F4FC20ED31EE41EF51E87EE93E0A0E092
:10127000B0E0C80ED91EEA1EFB1EC701B60128EE5B
:1012800033E040E050E00E94EA2ECA01B90128EEA6
:1012900033E040E050E00E94B82E1F910F91FF9084
:1012A000EF90DF90CF90BF90AF909F908F90089578
:1012B0008F3F910509F010F480E0089522E080301E
:1012C000920710F481E008958050934010F083E07D
:1012D000089582E00895CF92DF92FF920F931F93BB
:1012E000CF93DF93F82FEB016A01182F1695E0E0FA
:1012F00088819981D6018C938A819B8111968C93E8
:1013000011978C819D8112968C9312978E819F816B
:1013100013968C931397288139814A815B816C8164
:101320007D818E819F819295990F990F907C832F5B
:101330008370982B852F8370880F880F982B872FA9
:1013400083708295807F982B14969C9385E090E023
:10135000C80ED91E2896EF5F1E1750F6F0FF21C069
:10136000888199810E945809F82E8A819B810E9468
:101370005809182F8C819D810E945809082F8E8151
:101380009F810E945809F294FF0CFF0C70ECF72229
:101390001295107F1F29182B000F000F012BD6016B
:1013A0000C93DF91CF911F910F91FF90DF90CF9021
:1013B000089523E08032920718F420E030E026C040
:1013C00023E0883E920748F49C012F51334054E0BB
:1013D000369527955A95E1F719C027E0803D920789
:1013E00020F49C012C5D334011C028E0883992071D
:1013F00018F02FEF33E00AC09C01285C374044E02E
:10140000369527954A95E1F72D503C4FC90108952F
:101410009C013695279525753575821B930B9C018C
:101420003695279536952795237333738373937376
:10143000280F391FC901E4E096958795EA95E1F7F1
:10144000820F931F8F709F7021E031E0AC01429FAB
:10145000C001439F900D529F900D1124892F089534
:10146000882339F042980000419A0000429A000017
:1014700008954298000041980000429A00000895A3
:10148000429A000086B142980000817008950F933F
:101490001F93082F5C9A42985C9810E0802F807808
:1014A0000E94300A000F1F5F1830C1F742981F9149
:1014B0000F9108958F770E94470A08950F931F9305
:1014C000082F10E0802F80780E94300A000F1F5FE5
:1014D0001830C1F742981F910F9108950F931F93F1
:1014E000429880E000E0182F110F0E94400A810FFF
:1014F0000F5F0830C1F71F910F9108950E945A0A9B
:101500000E946E0A5C9A08951F93162F80680E94AD
:10151000470A812F0E945E0A5C9A1F9108951F93CB
:101520001091C7031827EEEBF3E0E80FF11D89E7F0
:1015300067850E94840A8DE3612F0E94840A82E4F9
:10154000612F0E94840A1F91089586E20E947E0AFC
:1015500008950F931F938C018CE1F80164810E9420
:10156000840A8DE1F80165810E94840A8EE1F80108
:1015700066810E94840A80E2F80167810E94840AE1
:1015800081E2F80160850E94840A82E2F8016185A7
:101590000E94840A83E2F80162850E94840A84E240
:1015A000F80163850E94840A85E2F80164850E943F
:1015B000840A8AE2F80165850E94840A8EE6F801B1
:1015C00066850E94840A8FE6F80167850E94840A76
:1015D00080E7F80160890E94840A81E7F801618947
:1015E0000E94840A82E7F80162890E94840A1F919E
:1015F0000F910895EF92FF920F931F93CF93DF9374
:101600007B018C01603028E372072CE982072CE112
:10161000920728F520E836E948E950E00E94EA2ED2
:10162000E9016897B90180E090E020E839E647E6F3
:101630005FEF0E94B82E6E0D7F1D801F911F22E06C
:10164000660F771F881F991F2A95D1F721E732E08F
:1016500040E050E00E94EA2E890180E421C020E0B1
:101660003DE241E351E00E94EA2EE9016897B901A9
:1016700080E090E020E033ED4EEC5EEF0E94B82E6B
:101680006E0D7F1D801F911F660F771F881F991F8A
:1016900021E732E040E050E00E94EA2E890180E636
:1016A0009E012F71622F680F85E70E94840A86E7EA
:1016B000612F0E94840A87E7602F0E94840ACDB7B9
:1016C000DEB7E6E00C944F2F9F92AF92BF92CF927D
:1016D000DF920F93DF93CF9300D000D0CDB7DEB76A
:1016E000982E83E00E947E0A8093E70384E00E94A4
:1016F0007E0A8093E80386E060E00E94840A87E027
:1017000061E00E94840A89E06FE70E94840A8AE00F
:1017100065E00E94840A8BE062E10E94840A8CE00A
:1017200065E10E94840A8DE06DEF0E94840A8EE0DC
:1017300060E00E94840A992019F084E193E008C0D7
:101740008091E50323E1829FC00111248B549D4FBA
:101750000E94A90A80E36CE80E94840A82E36FE099
:101760000E94840A83E362E40E94840A84E36AE0BC
:101770000E94840A85E36AE20E94840A86E36DE29D
:101780000E94840A87E364ED0E94840A88E360E093
:101790000E94840A89E360E00E94840A992049F04B
:1017A00055E7A52E51ECB52E51ECC52E5EEDD52E8C
:1017B00008C0A090C703B090C803C090C903D090E0
:1017C000CA030AE38D2D9927AA27BB2789839A8309
:1017D000AB83BC83802F69810E94840A802F8B5F3A
:1017E00069810E94840ADC2CCB2CBA2CAA240F5FBE
:1017F0000E3341F783E46FEF0E94840A84E46FEFB5
:101800000E94840A85E46FEF0E94840A86E46FEFE9
:101810000E94840A992019F08DE666E003C08DE6E7
:101820006091CB030E94840A89E760E00E94840AE9
:101830008AE76091CC030E94840A83E760E00E94FB
:10184000840A84E760E00E94840A992029F060EC11
:1018500072E98DEE99E108C06091C3037091C403F1
:101860008091C5039091C6030E94FA0A0F900F90D1
:101870000F900F90CF91DF910F91DF90CF90BF909D
:10188000AF909F90089587E061E00E94840A8EE700
:1018900064E20E94840A88E063E00E94840A88E08F
:1018A00060E00E94840A87E065E00E94840A85E087
:1018B00062E00E94840A83E00E947E0A8093E7032C
:1018C00084E00E947E0A8093E8030895582F409197
:1018D0008C04842F90E0FC01EF70F0709F012F5F6B
:1018E0003F4F64E0959587956A95E1F7281739078A
:1018F00051F0E458FB4F5083842F8F5F8F70407FEF
:10190000842B80938C0408951F920F920FB60F9230
:1019100011241F932F933F934F935F936F937F9364
:101920008F939F93AF93BF93CF93DF93EF93FF93E7
:10193000C0918600D09187002091CE043091CF04D1
:101940008091AD04882309F047C0CE01821B930B20
:101950009C0180919F0385FD02C03695279599E0F3
:10196000253C390708F1809147038630D0F08091FB
:1019700047038F3FB1F020E00EC0E22FF0E0EE0F02
:10198000FF1FDF01A255BB4F8D919C91E95DFC4F7C
:10199000918380832F5F80914703281770F3109203
:1019A000AC041092470318C082E02D3B380760F169
:1019B00080914703803140F510914703C9010E948F
:1019C000D909E12FF0E0EE0FFF1FE255FB4F9183A5
:1019D00080831F5F10934703D093CF04C093CE043E
:1019E000FF91EF91DF91CF91BF91AF919F918F9137
:1019F0007F916F915F914F913F912F911F910F9028
:101A00000FBE0F901F9018958FEF80934703E4CF80
:101A100083E0809380008AE98093810080919F0316
:101A200086FD05C0809181008064809381008FEFE6
:101A30009FEF909389008093880080916F0080626F
:101A400080936F0008956F3020F0869586958054BE
:101A500008958DE0689F802D11240895882319F43E
:101A600060E071E002C063E071E085E296E00E9410
:101A70006C2C0895A0E0B0E0E0E4FDE00C94312F80
:101A8000182F0E943F299B01AC0180911B0590916A
:101A90001C05A0911D05B0911E0569017A01C81AA7
:101AA000D90AEA0AFB0AD701C60189589341A04026
:101AB000B04010F010921A0520931B0530931C05BE
:101AC00040931D0550931E052091AD04822F815037
:101AD0008230E8F580911A05882309F44FC18130DE
:101AE00011F482E0BCC1803108F035C1E82FF0E08C
:101AF000E255FB4F10838F5F80931A05803109F008
:101B0000B0C1A0EBB4E0213039F41196EC911197FB
:101B1000E695E6958C9109C08D919C911197E92FDE
:101B2000E695E695E69596958795E03140F4F0E0E8
:101B300090E0EE0FFF1FE95DFC4F918380831092D0
:101B4000AC04129684E0AE3BB807E9F68AC12330B4
:101B500009F004C180911A05882321F41F3009F08F
:101B600080C10CC1883130F4E82FF0E0E355FB4F21
:101B7000108374C1883109F0EEC0112309F0EBC065
:101B8000C0E0D0E00BE010E0DE0163E0AA0FBB1F75
:101B90006A95E1F7C09FB001C19F700DD09F700D95
:101BA0001124FB01E255FB4F80812181922F977018
:101BB00095958795FD01EE0FFF1FE95DFC4F918321
:101BC0008083FB01E155FB4F308136953695369584
:101BD0002181422F4295440F407E842F832B2695EE
:101BE00026952695922F977095958795FD01EE0F76
:101BF000FF1FE75DFC4F91838083FB01E055FB4FA6
:101C0000808182958695869583704181942F990F66
:101C1000990F292F282B429546954695437082812E
:101C20008170880F880F382F342B35952795FD014B
:101C3000EE0FFF1FE55DFC4F31832083FB01EE5467
:101C4000FB4F308136952181422F47954427479598
:101C5000842F832B2695922F977095958795FD015C
:101C6000EE0FFF1FE35DFC4F91838083FB01ED547A
:101C7000FB4F308132953F702181422F4295407F4A
:101C8000842F832B22952F70922F9770959587958F
:101C9000FD01EE0FFF1FE15DFC4F91838083FB018F
:101CA000EC54FB4F8081881F8827881F4181942F27
:101CB000990F292F282B441F4427441F82818370AA
:101CC000880F382F342B35952795FD01EE0FFF1F18
:101CD000EF5CFC4F31832083FB01EA54FB4F3081E2
:101CE000369536952181422F4295440F440F407C12
:101CF000842F832B26952695922F977095958795FF
:101D0000AA0FBB1FFD01ED5CFC4F918380836954DA
:101D10007B4FFB0120812295269527704181342F2E
:101D2000330F330F330F832F822B942F9295969579
:101D3000977095958795AB5CBC4F11969C938E934D
:101D40002196C230D10509F01FCF8091C40483FDD4
:101D500002C01092AC0410921A0583C0243009F01E
:101D600080C040911A05442359F4183AB1F41092F6
:101D700022051092210588EA0E942A0881E06FC09E
:101D8000413019F410931F0504C0423031F4109310
:101D90002005812F0E942A085DC060912005262F12
:101DA00030E0220F331FE42FF0E0C90102968E17B6
:101DB0009F0734F0433268F7E555FB4F1083E9CFB6
:101DC0002D5F3F4F4091210550912205E217F30707
:101DD00049F4912F80E048275927509322054093DA
:101DE000210538C0812F90E04817590789F5809167
:101DF0001F05813069F5613118F080E1809320057D
:101E0000D09020054EEAE42E44E0F42E00E010E0ED
:101E10001BC0F701D081C0E0818190E08C2B9D2B0D
:101E200033E0969587953A95E1F70E94D909F80134
:101E3000EE0FFF1FE95DFC4F918380830F5F1F4F03
:101E400082E090E0E80EF91E0D1518F31092AC0434
:101E500010921A0580911A05882319F08F5F8093DC
:101E60001A05CDB7DEB7E8E00C944D2FFF920F9323
:101E70001F93CF93DF93182F092FF62E8EE30E9426
:101E8000840A212F302FC901EC0110E005C08FE733
:101E900069910E94840A1F5F1F15C8F385E064E002
:101EA0000E94840A83E00E947E0A8093E70384E014
:101EB0000E947E0A8093E8030E943F296093E90311
:101EC0007093EA038093EB039093EC0387E069E05F
:101ED0000E94840A81E080939803CDB7DEB7E5E0E5
:101EE0000C94502F0E94360F809198038130D9F4C2
:101EF0000E943F292091E9033091EA034091EB03CE
:101F00005091EC03621B730B840B950B605A76485F
:101F10008140904040F4E8CF85E296E067E071E0D0
:101F20000E946C2C0895809198038130A9F3089544
:101F300085E296E06EE70E94242E0895A0E0B0E0CE
:101F4000E4EAFFE00C94302F6C0185E296E06EE746
:101F50000E94242E760100E010E0C0E0D0E0B0E264
:101F6000BB2E0AC00830110521F49E012095F60110
:101F700020870894E11CF11CF7016081862F8D57A2
:101F8000823040F485E296E06DE70E94242EF7014E
:101F900060816B2585E296E00E94242E01151105D3
:101FA00051F0F70180819E01280F311DC32FDD27DD
:101FB000C20FD31FD0700F5F1F4F0930110591F66C
:101FC000CDB7DEB7E9E00C944C2FA9E0B0E0EBEE22
:101FD000FFE00C94372F382FE62F8091910490E08A
:101FE000019664E270E00E94D72E982F80939104AE
:101FF00088E9898380E18A83913071F0913028F0FB
:10200000923099F09330E1F416C085E08B8381EF34
:102010008C832F5F2D8317C09B8381EF8C8384E695
:10202000489FC00111249D830EC084E08B8381EF03
:102030008C833D8308C09B8381EF8C83ED8303C039
:102040000E94980F04C0CE0101960E949E0F29960F
:10205000E2E00C94532F0F931F93CF93DF93182F2D
:10206000092F85E296E06EE70E94242E212F302F63
:10207000C901EC0110E000E288818D57823040F404
:1020800085E296E06DE70E94242E88818027888370
:1020900085E296E069910E94242E1F5F193061F756
:1020A00085E296E06EE70E94242EDF91CF911F918A
:1020B0000F910895A9E0B0E0E0E6F0E10C94372F2D
:1020C000382F80919104882379F48EEF89833A83A5
:1020D0006B83842F90E0959587958C832D8319864B
:1020E00018861F821E822FC040918C04842F90E09E
:1020F0009C012F70307054E0959587955A95E1F7C3
:102100008217930721F18DEF89831A821B82DE01EA
:10211000149620E008C0E458FB4F80818D93405F07
:102120002F5F263069F0842F90E0FC0134E0F595B4
:10213000E7953A95E1F78F709070E817F90759F72E
:1021400040938C042A83CE0101960E942B1080912B
:10215000910490E0019666E070E00E94D72E809393
:1021600091042996E2E00C94532F9F92AF92BF9274
:10217000CF92DF92EF92FF920F931F93B82EA62E6D
:10218000D42EC22E902E0E943F297B018C0180917B
:102190007B0420918D0430918E0440918F045091E6
:1021A00090048823B1F0D801C701821B930BA40BC4
:1021B000B50B815E9E42A040B04020F12C2DDC1476
:1021C00008F42D2D8B2D6A2D422F292D0E94E50F0D
:1021D00011C0D801C701821B930BA40BB50B81530F
:1021E0009547A040B04070F08B2D6A2D4D2D2C2DC1
:1021F0000E945A10E0928D04F0928E0400938F0496
:10220000109390041F910F91FF90EF90DF90CF906B
:10221000BF90AF909F90089585E296E06091EE03A5
:102220000E94242E08951F93182F85E296E0612FB7
:102230000E94242E8091EE0381278093EE031F914C
:1022400008951F93192F0E941311812F0E941311BB
:102250001F910895DF92EF92FF920F931F93D82E54
:102260007B011092EE0305E216E0C80165EB0E94C7
:10227000242EC80162E60E94242E8D2D0E94131187
:10228000C7010E9421111F910F91FF90EF90DF90E5
:1022900008958EE060E00E94C4298FE061E00E9412
:1022A000C42980E161E00E94C42982E060E00E94CC
:1022B000C42984E061E00E94C4290895CF93DF938C
:1022C000EC01009741F186E061E00E94302A9E0116
:1022D00040E050E068E478EE81E090E00E940C2F4E
:1022E000C901DA018F3F9105A105B10531F028F050
:1022F0008FEF90E0A0E0B0E008C00097A105B10525
:1023000021F481E090E0A0E0B0E08093B300809100
:10231000B000806107C086E060E00E94302A8091B2
:10232000B0008F7E8093B000DF91CF910895A0E040
:10233000B0E0EDE9F1E10C942F2F8CE00E947E0AD1
:10234000882389F585E296E063E171E00E946C2CB8
:10235000439A299A80E00E94640B0E94430C4398A0
:10236000299821C085E296E00E94EB2D482F8091AC
:10237000AD04882321F0842F0E943A0D14C080916F
:102380001805E82FF0E031969F012F7130703197DA
:102390008091170590E02817390729F0E251FB4F8B
:1023A00040832093180585E296E00E94B12D892B89
:1023B000C9F680919803843009F08CC00E943F29AF
:1023C00060939C0470939D0480939E0490939F045B
:1023D000611571058105910561F481E090E0A0E04F
:1023E000B0E080939C0490939D04A0939E04B093CE
:1023F0009F048091A8049091A90481609093A904FE
:102400008093A80483E0809398038FE70E945A0A80
:10241000C5EED4E00E946E0A899304E0CE3ED00758
:10242000C9F74091D0048091E504282F30E0842F33
:1024300090E08227932786FF40C080E4482740939E
:10244000D004C90188739070C89709F510E014C0D2
:102450001F5F8091E603E12FF0E084FF06C0EB519F
:10246000FB4F80810E94660C07C0EB51FB4F85E259
:1024700096E060810E94242E212F30E08091E504B7
:1024800090E0877090708217930714F716C02F732F
:102490003070232B91F48091E6048093A004809106
:1024A000E7048093A2048091E8048093A3048091C0
:1024B000EB048093AA041092AB048091190581303B
:1024C00019F482E08093190580911905833011F485
:1024D000109219050E943F295B016C018091A404B0
:1024E0009091A504A091A604B091A7040097A1051E
:1024F000B105C9F0A6019501281B390B4A0B5B0BEE
:10250000DA01C901885B9B40A040B04060F00E94A6
:10251000A50A8093A1041092A4041092A50410921D
:10252000A6041092A7048EEB93E00E94E408209189
:1025300098043091990440919A0450919B0486012B
:102540007501E21AF30A040B150BE616F7060807E5
:10255000190708F4EFC0A0929804B0929904C092B1
:102560009A04D0929B04A8958091AC04883008F01E
:10257000D8C08091AC048F5F8093AC04E0909C0441
:10258000F0909D0400919E0410919F04E114F104C9
:102590000105110511F18EEB93E00E94E408AE18DD
:1025A000BF08C00AD10A6A157B058C059D0588F411
:1025B00080919F0384FD04C080ED97E00E945E112E
:1025C00010929C0410929D0410929E0410929F04FD
:1025D00004C080E090E00E945E119091D004907C55
:1025E0009093D00400911805109117050117B1F1CF
:1025F00080911905823091F590589093D0048EEB1C
:1026000093E00E94DA08893010F048E002C0482FB9
:10261000415030E013C03F5FA32FB0E0812F90E026
:10262000FC01E251FB4F2081FD01E053FB4F208371
:10263000A25FBA4F2C930196182F1F71341710F414
:10264000101749F710931705832F895C9091D004D8
:10265000892B8093D00430930E051AC02091190560
:102660002430D1F490910E05EFE0F5E0A1EDB4E057
:10267000292F30E02E0F3F1F02C081918D93E2176A
:10268000F307D9F7995C8091D004982B9093D004EC
:1026900083E08093190525C080919304823031F442
:1026A00091609093D004439A299A10C09093D004DB
:1026B00043982998222319F481E080931905809189
:1026C0001905833019F484E080931905F8948091FA
:1026D000E603877067E273E041ED54E00E946B0906
:1026E000789485B1846285B9809192040E948F0AA2
:1026F0008EEB93E00E94DA08682F80ED94E00E9450
:10270000360FE0919204EF5FE0939204E83131F0EC
:10271000F0E0E254FC4F8785882361F41092920424
:1027200009C08091AC04883011F4439A299A89E059
:102730008093AC048091E603887171F180919803D5
:10274000823051F58091A8049091A904880F991FB7
:102750009093A9048093A80483E0809398030E9437
:10276000430C0E943F296093A4047093A5048093B6
:10277000A6049093A704611571058105910561F484
:1027800081E090E0A0E0B0E08093A4049093A504E1
:10279000A093A604B093A7048091E60384FF1EC013
:1027A0008091A8049091A9048E7F0E94080A182F96
:1027B0008091A0046091AA040E94230D082F8091AB
:1027C000A104612F0E94230D282F8091A204609103
:1027D000A304402F009199030E94B51085B18B7D11
:1027E00085B9809193048130C9F0813020F0823026
:1027F00009F03FC033C087E00E94632A892BC9F5E6
:1028000081E0809393040E94312960939404709333
:10281000950480939604909397042BC087E00E94C0
:10282000632A892B21F50E9431292091940430914B
:1028300095044091960450919704621B730B840B8E
:10284000950B695E73408040904098F082E08093E1
:10285000930480ED97E00E945E110BC087E00E9418
:10286000632A892B31F080E090E00E945E11109283
:102870009304CDB7DEB7EAE00C944B2F86E061E01D
:102880000E94C42986E060E00E94302A82E08093A2
:10289000B00085E08093B10083E061E00E94C4292C
:1028A00083E060E00E94302A08951F93182F0E9451
:1028B0003F2960938D0470938E0480938F049093CE
:1028C000900410937B04112329F440E855E260E062
:1028D00070E004C040E051EE60E070E085E296E018
:1028E0000E942A2D1F910895ACE1B0E0EAE7F4E1DF
:1028F0000C942F2F0E943F297B018C0181E00E94C4
:10290000640BA4E7AA2E6E010894C11CD11CF3E04D
:10291000BF2EA982C60161E00E94720FB092980397
:102920000E94430C6AEF70E080E090E00E9465290D
:1029300080919803833009F07DC085E296E00E9483
:10294000B12D892B09F076C00E943F296E197F09AD
:10295000800B910B6058734C894C914008F06AC011
:10296000D8CF8FE70E945A0A0E946E0A843509F078
:102970005CC089830E946E0A182F00E010937A04CD
:10298000009379040E946E0A080F111D10937A04B7
:10299000009379040E946E0A809378040E946E0A64
:1029A00080937704813108F040C0FF2407C00E9463
:1029B0006E0A095A1B4FF8018083F3940F2D10E023
:1029C0008091770490E0880F991F0817190778F312
:1029D00080E78983CE01019661E00E94720F83E057
:1029E000809398030E94430C62E370E080E090E0E3
:1029F0000E946529809198038330A9F08FE70E9497
:102A00005A0A0E946E0A803581F4898303EA13E032
:102A10000E946E0AF80181938F01F3E00E3B1F07BD
:102A2000B9F781E003C082E001C083E06C96EAE080
:102A30000C944B2F80919803833009F092CFF3CF01
:102A400083E00E947E0A8093E70384E00E947E0A6E
:102A50008093E80387E061E00E94840A6AE070E006
:102A600080E090E00E9465290E94430C00000895D8
:102A70000F931F93082F19C0439A299A64E670E0B8
:102A800080E090E00E9465294398299864E670E010
:102A900080E090E00E9465291F5F101768F36CE2E8
:102AA00071E080E090E00E94652910E0F6CF482FA9
:102AB000392F25E00DC0F999FECF1FBA842F932F2F
:102AC00092BD81BD60BD0FB6F894FA9AF99A0FBE17
:102AD000215059F0F999FECF842F932F92BD81BDDB
:102AE000F89A80B5681739F7089582E00E94381582
:102AF0000895A0E0B0E0EFE7F5E10C94282F482E10
:102B0000562EEE24FF2488249924C0E0D0E0CC2463
:102B1000DD2436E3332E04C055245394CC24DD2425
:102B2000442069F480919903839DE00111242AE9EE
:102B3000E22E23E0F22E99E0892E912C1DC021E097
:102B4000421671F480919903839DE00111242B9624
:102B50008EEBE82E83E0F82E09E2802E912C0CC03B
:102B600032E0431649F419E9E12E13E0F12EB1E009
:102B70008B2E912CC8EDD0E03E016C0C7D1C109288
:102B8000220510922105E3011BC0552059F4F99943
:102B9000FECFD2BDC1BDF89A80B5F701E00FF11F9D
:102BA000808307C0F701E00FF11FCE0160810E9412
:102BB00057150E0D1F1DF80180810E942A082196CD
:102BC0009E012619022F10E008151905F0F2CE011A
:102BD0005520D9F4F999FECFD2BDC1BDF89A20B5E0
:102BE000F999FECF2196D2BDC1BD2197F89A80B543
:102BF00090E0B22EAA248A299B29209121053091A8
:102C000022052817390759F487CF219660912205AC
:102C10000E945715CE01609121050E94571580E052
:102C200091E0C80ED91E91E0C91693E0D90608F4C8
:102C300077CF852DCDB7DEB7E1E10C94442F80E04E
:102C400061E00E94791581E061E00E9479150895A4
:102C500080E060E00E947915882331F081E060E037
:102C60000E947915882331F40E948C080E9447083D
:102C70000E941F16089582E061E00E947915089570
:102C800082E060E00E94791580919903843020F001
:102C9000109299030E943B1608951F93182F0E94CB
:102CA000401680919903811731F0143020F410936D
:102CB00099030E943B161F9108951092550485E6D2
:102CC000E0EFF3E0DF011D928A95E9F708951F9385
:102CD000182F8F3711F08830E1F5E0915504EE237D
:102CE00009F455C0E150E0935504F0E0E051FC4F89
:102CF000108285E296E06DE00E94242E10E00AC06A
:102D0000E12FF0E0E051FC4F85E296E060810E9407
:102D1000242E1F5F80915504181790F385E296E0EA
:102D200060E20E94242E85E296E06DE00E94242E4F
:102D300010E00AC0E12FF0E0E051FC4F85E296E0A0
:102D400060810E94242E1F5F80915504181790F314
:102D50001CC08B3119F40E945D161FC08D30E9F044
:102D60008A30D9F080915504843688F485E296E063
:102D7000612F0E94242E80915504E82FF0E0E0514D
:102D8000FC4F10838F5F8093550480E007C085E27D
:102D900096E067E00E94D82AF8CF81E01F9108955D
:102DA0001F93CF93DF93CDECD3E010E03BC085E2DF
:102DB00096E062E271E00E94692C85E296E0612F64
:102DC0004AE050E00E94E62B85E296E06FE271E077
:102DD0000E94692C699170E080E090E02091CC0322
:102DE00030E040E050E00E94B82E20E137E240E0C1
:102DF00050E00E94B82EDC01CB014091C3035091FA
:102E0000C4036091C5037091C603480F591F6A1F20
:102E10007B1F85E296E02AE030E00E94AD2B1F5F29
:102E2000183119F08881882311F6DF91CF911F9115
:102E30000895EF92FF920F931F93882339F485E250
:102E400096E066E67AE00E94F62A3BC090E00E9497
:102E5000A10824E630E040E050E00E94EA2E122F64
:102E6000032FF42EE52E622F732F842F952F2AE047
:102E700030E040E050E00E94EA2E85E296E0BA01A0
:102E8000A9012AE030E00E949E2B85E296E06EE2E6
:102E90000E94D82A612F702F8F2D9E2D2AE030E0BE
:102EA00040E050E00E94EA2EAB01BC0185E296E0D2
:102EB0002AE030E00E949E2B85E296E063E70E94C4
:102EC0000A2B1F910F91FF90EF900895FF920F939F
:102ED0001F93CF93DF9385E296E06CE57AE00E9442
:102EE000B72A8091A303813041F485E296E063E440
:102EF0007AE00E94F62AFF2466C0823029F485E237
:102F000096E06CE27AE0F5CF8430A9F785E296E0AE
:102F100068E17AE0EECFCF2DD0E0C930D1051CF0CA
:102F20006F2D685C02C06F2D6F5C85E296E00E9499
:102F3000D82A85E296E060E17AE00E94B72ABE01D5
:102F40006F5F7F4F85E296E04AE050E00E94422C9E
:102F500085E296E065E07AE00E94B72A8E010D5581
:102F60001C4FD8011196EC91E032F8F485E296E01E
:102F700068EF79E00E94B72AF8018181803130F052
:102F800085E296E063E371E00E94692CCD55DC4F49
:102F9000698170E06F7070706F5F7F4F85E296E0BF
:102FA0004AE050E00E94552C0DC0F0E0EF70F07048
:102FB000EE0FFF1FE85BFC4F6081718185E296E0B8
:102FC0000E946C2CF39480917804F81608F4A3CF37
:102FD00085E296E06DED79E00E94B72A8091BB030F
:102FE0000E94191785E296E062EC79E00E94B72A08
:102FF0008091BC030E94191785E296E067EA79E0A8
:103000000E94B72A8091BD030E94191785E296E0BD
:103010006CE879E00E94B72A4091B3035091B40361
:103020006091B5037091B6034115510561057105B5
:1030300039F185E296E02AE030E00E94AD2B85E28E
:1030400096E069E579E00E94B72A8091B7030E9473
:10305000D408AB01BC0185E296E02AE030E00E9492
:10306000AD2B85E296E065E379E00E94B72A85E220
:1030700096E06091B8034AE050E00E94F82B06C049
:1030800085E296E06CE279E00E94F62A85E296E01D
:103090006FE079E00E94B72A6091B9037091BA039A
:1030A00085E296E04AE050E00E94D22B85E296E06D
:1030B00062EF78E00E94B72A6091B203603150F469
:1030C00070E06F5F7F4F85E296E04AE050E00E943B
:1030D000552C06C085E296E069EE78E00E94F62A5B
:1030E00085E296E06CEC78E00E94B72A8091B1030B
:1030F00080FD03C065E371E002C069E371E085E231
:1031000096E00E946C2C85E296E06FEA78E00E94DF
:10311000B72A8091B10382700E942E0D85E296E05D
:1031200060E978E00E94B72A8091B10384700E9420
:103130002E0D85E296E061E778E00E94B72A809143
:10314000B10388700E942E0DCDB7DEB7E5E00C9478
:10315000502F1F93CF93DF9385E296E060EB7BE0E7
:103160000E94B72A4091C3035091C4036091C503E4
:103170007091C60385E296E02AE030E00E94AD2B14
:1031800085E296E06AE97BE00E94B72A4091C70396
:103190005091C8036091C9037091CA0385E296E01B
:1031A00020E130E00E94AD2B85E296E064E87BE010
:1031B0000E94B72A85E296E06091CB034AE050E096
:1031C0000E94F82B85E296E06EE67BE00E94B72A2B
:1031D00085E296E06091CC034AE050E00E94F82B33
:1031E00085E296E068E57BE00E94B72ACDECD3E06B
:1031F00010E012C0112331F085E296E06DE371E03A
:103200000E94692C85E296E069914AE050E00E94B4
:10321000E62B1F5F183119F08881882359F785E262
:1032200096E00E94E02A85E296E062E47BE00E945C
:10323000B72A85E296E06091E5034AE050E00E94FB
:10324000F82B85E296E06DE27BE00E94B72AE091E0
:10325000E603F0E0E770F070EE0FFF1FE859FC4F57
:103260006081718185E296E00E946C2C85E296E097
:1032700068E17BE00E94B72A8091E60390E08871C4
:1032800090708830910589F0893091051CF4892B64
:1032900039F01BC08031910569F04897B1F40FC037
:1032A00085E296E06FE07BE00EC085E296E063E0A9
:1032B0007BE009C085E296E06DEF7AE004C085E22C
:1032C00096E063EF7AE00E94F62A85E296E06FEDE1
:1032D0007AE00E94B72A4091BF035091C0036091E9
:1032E000C1037091C20385E296E02AE030E00E94BB
:1032F000AD2B85E296E066EC7AE00E94B72A8091D9
:103300009F0380710E942E0D85E296E06DEA7AE0BF
:103310000E94B72A80919F0380740E942E0D85E23F
:1033200096E064E97AE00E94B72A80919F03807258
:103330000E942E0D85E296E067E77AE00E94B72AA8
:103340008EEB93E00E94E408AB01BC0185E296E0BD
:103350002AE030E00E949E2B85E296E062E77AE068
:103360000E94B72A8EEB93E00E94E4089B01AC0117
:1033700060E472E48FE090E00E94EA2E85E296E03D
:10338000BA01A9012AE030E00E949E2B85E296E076
:103390006FE67AE00E94F62ADF91CF911F9108959F
:1033A000EF92FF920F931F937C0105E216E0C80194
:1033B0006F2D70E04AE050E00E94C12BC8016EE220
:1033C0000E94D82AB701E4E076956795EA95E1F77F
:1033D0006F707070C8014AE050E00E94C12BC801B4
:1033E0006EE20E94D82A8FE0E822FF24C801B701CC
:1033F0004AE050E00E94C12B1F910F91FF90EF9087
:1034000008950F931F93CF93DF932091EF032F3FE6
:10341000A9F585E296E061EF75E00E94B72A82E6A1
:1034200093E00E94D01985E296E060ED75E00E947D
:10343000B72A8091790490917A040E94D01985E28C
:1034400096E06DE975E00E94F62A85E296E06AE76B
:1034500075E00E94F62A85E296E062E675E00E9439
:10346000F62A85E296E06DE375E00E94F62A85E291
:1034700096E00E94E02A0E94661769C012160CF0BE
:1034800066C0332727FD30958091780490E082173D
:1034900093070CF45CC085E296E068E275E00E9458
:1034A000B72A6091EF03772767FD709585E296E074
:1034B0004AE050E00E94552C85E296E06DEF74E002
:1034C0000E94B72A08E210E03AC0C12FD0E0CC0F2A
:1034D000DD1FC95ADB4F288130E08091EF03992727
:1034E00087FD909501972817390741F585E296E009
:1034F0006FE371E00E94692C85E296E0602F4AE05C
:1035000050E00E94E62B85E296E063E471E00E94C1
:10351000692CE981F0E0EF70F070EE0FFF1FE85BBF
:10352000FC4F6081718185E296E00E94692C85E202
:1035300096E067E471E00E94692C0F5F1F5F809145
:103540007704181710F285E296E00E94E02ADF91D6
:10355000CF911F910F910895ACE1B0E0E2EBFAE159
:103560000C94312F282F8091EF038F3F09F042C137
:10357000822F90E0FC013A97EF36F10508F033C155
:10358000EC5CFF4F0C945E2F85E296E069E471E0FD
:10359000AEC085E296E069E471E00E946C2C1CC12B
:1035A00085E296E065E571E00E946C2C85E78983F1
:1035B000DE011296E3EAF3E08BE101900D92815077
:1035C000E1F7CE0101966CE10E94720F0E94430C5C
:1035D00083E08093980368EC70E080E090E00E94C4
:1035E000652980919803843009F0FDC08FE70E941F
:1035F0005A0A0E946E0A8983853509F0F4C085E273
:1036000096E06FED74E00E94F62A85E296E061ECA8
:1036100074E00E94F62A85E296E063EA74E0ACC0AA
:1036200085E296E06DE671E00E946C2C89E6898364
:10363000CE01019661E00E94720F0E94430C83E06C
:103640008093980368EC70E080E090E00E94652928
:1036500080919803843009F0C6C08FE70E945A0A0F
:103660000E946E0A89838E010E5F1F4F2DE1E22EAC
:10367000F12CEC0EFD1E0E946E0AD8018D938D0177
:10368000AE15BF05C1F7A3EAB3E0FE0132968BE1A8
:1036900001900D928150E1F78981893409F0A3C02E
:1036A00085E296E065E874E00E94F62A85E296E0FD
:1036B00067E674E00E94F62A85E296E069E474E029
:1036C0005BC085E296E067E871E00E946C2C8EEFAB
:1036D0008093EF0388C020522750922F90538091FF
:1036E0007804891738F485E296E066E971E00E9473
:1036F0006C2C79C09093EF036FC084E18093EF034B
:1037000085E296E062E174E037C085E18093EF03E3
:1037100085E296E06BED73E02FC086E18093EF03C6
:1037200085E296E064EA73E027C087E18093EF03C7
:1037300085E296E06AE573E01FC088E18093EF03BD
:1037400085E296E069E473E017C089E18093EF03B6
:1037500085E296E065E373E00FC08AE18093EF03B2
:1037600085E296E060E273E007C08BE18093EF03AF
:1037700085E296E068EF72E00E94F62A34C085E2A6
:1037800096E06EED72E00E94F62A8091B10391E01E
:103790001DC085E296E068EC72E00E94F62A8091F6
:1037A000B10392E013C085E296E063EB72E00E9401
:1037B000F62A8091B10394E009C085E296E068E9B9
:1037C00072E00E94F62A8091B10398E089278093E5
:1037D000B1038FEF8093EF030E94011A04C085E2CA
:1037E00096E00E94EB2D85E296E00E94B12D892B98
:1037F000B1F762C1822F0E946716882309F45CC169
:1038000080915504882321F48FEF8093EF034CC1FE
:1038100080EF93E060E070E040E050E00E949C06A2
:103820009B01AC016091EF03862F992787FD90954E
:10383000A92FB92FFC013197EB31F10508F024C114
:10384000ED55FF4F0C945E2FE62FFF27E7FDF09517
:103850008091780490E08E179F070CF415C1DA016F
:10386000C9010197A109B1098097A105B10548F0E7
:1038700098E2F92E00E010E06F010894C108D10829
:1038800025C0ED55FC4F822F81508083E5C0612F0C
:1038900070E0660F771F695A7B4FFB01808190E0D3
:1038A0008C159D0591F48F2D90E0A0E0B0E082177B
:1038B0009307A407B50741F4F601ED55FC4FDB0172
:1038C00011968C91818301E0F3941F5F80917704BE
:1038D0001817E8F2BFC02F3F31054105510511F01F
:1038E00008F0D2C02093BB03B7C02F3F310541057C
:1038F000510511F008F0C8C02093BC03ADC02F3FA4
:1039000031054105510511F008F0BEC02093BD03FB
:10391000A3C08091F0038062803719F581EF93E0B6
:1039200060E070E040E050E00E949C069B01AC012A
:10393000DC01CB010197A109B1090897A105B105E7
:1039400008F0B5C0CA01B90124ED30E340E050E011
:103950000E94B82E9B01AC012A5E3C4A4A46554E55
:1039600024C0863611F581EF93E060E070E040E01E
:1039700050E00E949C069B01AC01DC01CB01019749
:10398000A109B1090797A105B10508F090C0CA01C6
:10399000B90128EA31E640E050E00E94B82E9B01D0
:1039A000AC01245E3C434E46544E21153105410581
:1039B000510561F0DA01C9018054914EAD49B84119
:1039C0008158904FAA4FB24008F05EC02093B303D5
:1039D0003093B4034093B5035093B6033DC02F3FDB
:1039E00031054105510511F008F04EC02093B70391
:1039F00033C0DA01C9010197A109B1098F3F9105CF
:103A0000A105B10508F040C02093B80325C0DA0134
:103A1000C901845C9940A040B0408D549D41A040B4
:103A2000B04030F43093BA032093B90301E001C0F1
:103A300000E0211531054105510511F48FEF07C054
:103A4000213131054105510528F4822F81508093A1
:103A5000B20302C00023C1F0809156048823D1F440
:103A60008091C7039091C803A091C903B091CA0384
:103A70000196A11DB11D8093C7039093C803A09325
:103A8000C903B093CA0306C085E296E068EA71E014
:103A90000E946C2C0E945D168FEF8093EF0385E2ED
:103AA00096E06AE00E940A2B0E94011A05C021E0FC
:103AB00030E040E050E07ECF6C96E8E00C944D2F73
:103AC00085E296E06CE472E00E94F62A85E296E0D8
:103AD00064E372E00E94F62A85E296E00E94B12D2E
:103AE000892B31F085E296E00E94EB2D0E94AC1A02
:103AF0000E947414823019F0833069F405C085E2A5
:103B000096E066E172E004C085E296E06FEF71E056
:103B10000E94F62A08958FEF8093EF0310925604C7
:103B20000E94011A0CC085E296E00E94B12D892BFB
:103B300031F085E296E00E94EB2D0E94AC1A809154
:103B4000EF038E3F81F708958091EF03992787FD5A
:103B50009095A92FB92FFC013196EB30F10508F0B3
:103B600074C0E254FF4F0C945E2F85E296E064E649
:103B700078E00E94F62A82E693E00E94D01985E25E
:103B800096E06CE478E00E94F62A85E296E067E22F
:103B900078E00E94F62A85E296E06DEF77E00E94D9
:103BA000F62A85E296E06CED77E00E94F62A85E23F
:103BB00096E06FEA77E00E94F62A85E296E069E8EF
:103BC00077E00E94F62A85E296E065E677E00E94BB
:103BD000F62A85E296E06EE377E00E94F62A85E217
:103BE00096E00E94E02A0E94A9182FC085E296E084
:103BF00061E277E028C085E296E06CEF76E023C0D2
:103C000085E296E067EE76E01EC085E296E068EC1D
:103C100076E019C085E296E064E876E014C085E2BB
:103C200096E06FE676E00FC085E296E06AE576E022
:103C30000E94F62A85E296E064E176E004C085E21F
:103C400096E06EEF75E00E94F62A6AE070E080E090
:103C500090E00E94652904C085E296E00E94EB2D69
:103C600085E296E00E94B12D892BB1F70895A2E27A
:103C7000B0E0EDE3FEE10C94272F8E010F5F1F4FA4
:103C800080E1D8011D928A95E9F785E296E066EC1D
:103C900071E00E946C2C0E94201520E431EE4DE969
:103CA00058E12F8F38A349A35AA380EC91EDA8E9DE
:103CB000BBE18B8F9C8FAD8FBE8F24EF31E040E056
:103CC00050E02F8B388F498F5A8F60E5C62E63ECFA
:103CD000D62EE12CF12C50E4452E51EE552E5DE907
:103CE000652E58E1752E88249924540133241E8AA8
:103CF0001D8A198A1A8A1B8A1C8AFFC085E296E0EF
:103D00000E94EB2D8434B9F0853430F48332B9F15C
:103D10008C3209F0CCC044C0833509F0C8C02F8D67
:103D200038A149A15AA1C901DA012C013D01882419
:103D300099245401E2C085E296E064E40E94D82A06
:103D400085E296E040E451EE6DE978E12AE030E06A
:103D50000E940C2C85E296E06CE20E94D82A85E253
:103D600096E040EC51ED68E97BE12AE030E00E940A
:103D70000C2C85E296E06CE20E940A2BBEC01982F0
:103D80001A821B821C821D821E821F82188619863F
:103D90001A861B861C861D861E861F86188A3AC0B8
:103DA000339434E0331609F0A8C069817A818B819D
:103DB0009C8128EE33E040E050E00E94B82E6F8FE7
:103DC00078A389A39AA36D817E818F8198850E94B3
:103DD000B82E6B8F7C8F8D8F9E8F89859A85AB8552
:103DE000BC858F8B988FA98FBA8F6D857E858F85C7
:103DF00098890E94B82E6B017C0190E2C9169EE45E
:103E0000D90690E0E90690E0F90630F48CE162E32F
:103E10000E94840A332471C0A0E3CA16A5E7DA061B
:103E2000A0E0EA06A0E0FA0618F48CE162E2F0CF26
:103E3000B0E4CB16BCE9DB06B0E0EB06B0E0FB0675
:103E400018F48CE166E2E4CFE0E5CE16E3ECDE06A2
:103E5000E0E0EE06E0E0FE0618F48CE162E1D8CF87
:103E6000F0E6CF16FAEEDF06F0E0EF06F0E0FF0630
:103E700018F48CE165E1CCCF20E7C21621E1D2062F
:103E800021E0E20620E0F20618F48CE161E0C0CF08
:103E900030EAC31636E8D30631E0E30630E0F30635
:103EA00018F48CE163E0B4CF8CE165E0B1CF40ED74
:103EB000242E280E49E0421500F1032D10E0000FDA
:103EC000111F000F111F81E090E08C0F9D1F080F44
:103ED000191FD8016D917D918D919C912AE030E060
:103EE00040E050E00E94B82E620D711D811D911DB1
:103EF000F801608371838283938385E296E00E9458
:103F0000B12D892B09F0FACE81149104A104B104DA
:103F100089F4C301B2010E94FA0A61E070E080E016
:103F200090E00E946529FFEFFE8B1D8A198A1A8A8C
:103F30001B8A1C8A2F89388D498D5A8D82169306CB
:103F4000A406B506E0F40E94A50A29893A894B899E
:103F50005C89280F311D411D511D298B3A8B4B8BDC
:103F60005C8B3D89381708F48D8B4E89841708F4D3
:103F70008E8B0894811C911CA11CB11C56C0C301DE
:103F8000B20128EE33E040E050E00E94EA2E85E2E4
:103F900096E0BA01A9012AE030E00E949E2B85E25A
:103FA00096E06CE20E94D82A85E296E06D894AE0AC
:103FB00050E00E94E62B85E296E06CE20E94D82A4F
:103FC00069897A898B899C89A50194010E94EA2ECE
:103FD00085E296E0BA01A9012AE030E00E949E2B1A
:103FE00085E296E06CE20E94D82A85E296E06E892E
:103FF0004AE050E00E94E62B85E296E06CE20E94E7
:104000000A2B4C0C5D1C6E1C7F1C8B8D9C8DAD8D0A
:10401000BE8D84159505A605B70520F44F8C58A0D4
:1040200069A07AA08824992454012F8D38A149A130
:104030005AA1285E33404040504009F05ECFA2961E
:10404000E2E10C94432FAAE5B0E0E9E2F0E20C943F
:10405000332F8B017A018B3009F425C18C3040F568
:10406000853009F484C0863080F4823009F459C068
:10407000833020F4813009F044C242C0833009F417
:1040800061C0843009F03DC265C0883009F49DC02C
:10409000893038F4863009F486C0873009F031C29F
:1040A0008CC0893009F499C08A3009F02AC2C9C08D
:1040B000893609F476C18A3680F4863609F421C13E
:1040C000873620F4853609F01CC202C1873609F410
:1040D00031C1883609F015C235C18C3609F4B8C132
:1040E0008D3638F48A3609F467C18B3609F009C277
:1040F000A3C18D3609F4E0C1873C09F002C2F4C1C6
:1041000081E069E270E00E942A110EEB13E0F801F1
:1041100081918F010E941311F3E0073E1F07B9F749
:10412000F8C182E06BE170E00E942A1103EA13E01B
:10413000F80181918F010E941311F3E00E3B1F07DC
:10414000B9F7E7C183E061E070E00E942A110E94A4
:104150007414DDC184E061E070E00E942A1181E006
:104160000E9413110E940C110E94371ED4C160914D
:10417000770470E0660F771F85E00E942A1100E047
:1041800010E008C0F801E95AFB4F80810E9413112A
:104190000F5F1F4F8091770490E0880F991F0817D9
:1041A000190780F3B6C186E062E070E00E942A1130
:1041B00082E693E00E942111ACC187E061E070E0EB
:1041C0000E942A1180917804A2C188E061E070E029
:1041D0000E942A11809199039AC186E68983CE01B3
:1041E000019661E00E94720F0E94430C83E080936D
:1041F000980368EC70E080E090E00E94652980916F
:1042000098038430E1F48FE70E945A0A0E946E0AF4
:104210008983863471F489E060E270E00E942A119B
:1042200010E00E946E0A0E9413111F5F1032C9F73E
:1042300070C189E061E070E00E942A11BBC089E092
:1042400061C18AE069E070E00E942A1110929A032D
:1042500080918F05882351F080919F039091A00356
:10426000A091A103B091A203806809C080919F032F
:104270009091A003A091A103B091A2038F778093A6
:104280009F039093A003A093A103B093A2030AE914
:1042900013E0F80181918F010E941311F3E0033ABA
:1042A0001F07B9F736C18BE060E270E00E942A1167
:1042B000F89400E010E0F801E95DFC4F80810E9475
:1042C00013110F5F1F4F00321105A9F7789421C118
:1042D00085E661E070E00E942A110932110509F0BB
:1042E00015C120E030E0F901E254FC4FD701A20FE4
:1042F000B31F8C9180832F5F3F4F2932310599F78F
:1043000059C086E661E070E00E942A110B31110568
:1043100009F0FCC020E030E0F901ED55FC4FD70179
:10432000A20FB31F8C9180832F5F3F4F2B3131053C
:1043300099F740C087E661E070E00E942A110E9470
:104340001F1638C088E661E070E00E942A1185E7F8
:104350008A83DE011396E3EAF3E08BE101900D928C
:104360008150E1F7CE0102966CE10E94720F0E942B
:10437000430C83E08093980360E273E080E090E078
:104380000E94652980919803843009F0BFC08FE7AF
:104390000E945A0A0E946E0A8A83853509F0B6C0C7
:1043A00009C089E661E070E00E942A110E94470876
:1043B0000E948C0881E0ABC08AE661E070E00E9458
:1043C0002A1189E68E8FCE014E9661E00E94720F0F
:1043D0000E94430C83E08093980360E273E080E0E6
:1043E00090E00E94652980919803843009F08EC086
:1043F0008FE70E945A0A0E946E0A8E8F8E01015E1C
:104400001F4F7AE3E72EF12CEC0EFD1E0E946E0A80
:10441000F80181938F01EE15FF05C1F7A3EAB3E020
:10442000FE017F968BE101900D928150E1F78E8D18
:10443000893409F06BC0BECF8BE661E070E00E946A
:104440002A11F70180810E944D160E942816B2CFD2
:104450008CE661E070E00E942A110032110571F4CF
:1044600087E68AAFDE01DB96F70180E201900D92CC
:104470008150E1F7CE01CA9661E205C087E48AAFB8
:10448000CE01CA9661E00E94720F0E94430C83E045
:10449000809398036CE474E080E090E00E946529CA
:1044A00080919803843091F58FE70E945A0A0E9408
:1044B0006E0A873459F57ECF8DE661E070E00E9488
:1044C0002A110930110511F520E030E0F901E65616
:1044D000FC4FD701A20FB31F8C9180832F5F3F4FFA
:1044E0002930310599F766CF87EC61E070E00E94D2
:1044F0002A1181E00E9413110E940C111092ED0309
:104500000AC08AEC61E070E00E942A1180E00E94FB
:1045100013110E940C11C65ADF4FE6E00C944F2F86
:10452000A0E0B0E0E6E9F2E20C942F2F34E0A32EF5
:1045300026E0B22E95E0C92E03E215E084E6D82EDF
:10454000B2E0EB2EA3E0FA2EA1C085E296E00E9435
:10455000EB2D982F80938E0580918D05833021F16E
:10456000843028F4813099F08230B8F409C0853065
:1045700009F448C0853020F1863009F087C05FC05B
:10458000953B09F083C081E080938D057FC0923612
:1045900009F07AC0E0928D0579C090938C059093D4
:1045A0008B05F0928D0572C09093890510928A0553
:1045B00080918B05892780938B05A0928D0566C01D
:1045C000D92FC0E02091890530918A052C2B3D2BF5
:1045D00030938A052093890580918B0589278093E4
:1045E0008B05C0928D052536310508F44FC08CEC43
:1045F00061E070E00E942A1181E00E9413110E9484
:104600000C1142C02091870530918805F901ED5DBC
:10461000FA4F908380918B05892780938B052F5FBC
:104620003F4F3093880520938705809189059091AD
:104630008A052817390750F1B0928D0527C080915F
:104640008B05891759F460918705709188058091D1
:104650008C0543E255E00E9423200DC08BEC62E004
:1046600070E00E942A1180918C050E9413118091A4
:10467000EE030E941311F8018D2D11928A95E9F72E
:10468000109288051092870510928D0585E296E0BC
:104690000E94B12D892B09F058CFCDB7DEB7EAE0E3
:1046A0000C944B2F81E08093ED0308C085E296E0E7
:1046B0000E94B12D892B11F00E9490228091ED0370
:1046C0008823A1F70895A0E0B0E0E9E6F3E20C94B6
:1046D000322F0E943F296115710581059105C9F3AB
:1046E0000E9493061092C7031092C8031092C90348
:1046F0001092CA03DD24E090C703F090C803009134
:10470000C9031091CA03102F0F2DFE2CEE240E9416
:104710008E062FEF30E040E050E00E940C2FE60EB6
:10472000F71E081F191FE092C703F092C8030093F9
:10473000C9031093CA03D39444E0D416E1F6CDEC38
:10474000D3E000E010E040E1E42E47E2F42E4EC05A
:104750000F5F19F40E9447084DC00E948E0622E3A5
:1047600030E040E050E00E940C2F6F5FEDECF3E092
:1047700090E004C08191861759F39F5F9117D0F3A1
:104780008091CC0390E08E9D90018F9D300D9E9D79
:10479000300D1124862F90E0AC01249FC001259F8D
:1047A000900D349F900D1124AA2797FDA095BA2F44
:1047B0002091C3033091C4034091C5035091C603B7
:1047C000820F931FA41FB51F20919B0330919C0360
:1047D00040919D0350919E03281739074A075B07B4
:1047E00008F4B6CF69931F5F183121F088818823C0
:1047F00009F0AECFCDB7DEB7E7E00C944E2F1F9394
:104800001091EF031F3F09F0F1C0893409F467C02C
:104810008A3428F5883309F479C0893368F4803301
:1048200009F486C0813308F06FC08B3109F44DC0A4
:10483000813209F0D5C03DC0813409F49AC0823478
:1048400038F4893309F472C0803409F0C9C031C02A
:10485000823409F4A1C0863409F0C2C052C0823645
:1048600009F49AC0833690F4883579F1893538F4A3
:10487000823509F43FC0833509F0B2C01FC08A35C4
:1048800009F4A9C0813609F0ABC073C0823791F139
:10489000833730F48636A9F1893609F0A1C01FC0EC
:1048A000883799F08A3709F496C0833709F098C0A1
:1048B00005C085E296E069E471E019C00E941F1608
:1048C00085E296E063ED71E006C00E94281685E25D
:1048D00096E06DEE71E00E946C2C8EEF7FC00E941E
:1048E00047080E948C0885E296E06CE072E00E9426
:1048F0006C2C76C00E94632385E296E065E272E04C
:10490000F6CF0E94D0166CC0805368C085E296E056
:104910006CEE71E00E94F62A9091E603892F885F81
:104920008871977E892B8093E60320C089E056C06A
:1049300085E296E069ED71E00E94F62A80919F037E
:104940009091A003A091A103B091A20320E130E0D7
:1049500040E050E082279327A427B52780939F0348
:104960009093A003A093A103B093A2031093EF032D
:1049700037C085E296E063EC71E00E94F62A8091F0
:104980009F039091A003A091A103B091A20320E402
:1049900030E040E050E012C085E296E062EB71E06A
:1049A0000E94F62A80919F039091A003A091A103F9
:1049B000B091A20320E230E040E050E0822793274C
:1049C000A427B52780939F039093A003A093A103EE
:1049D000B093A20302C00E94601D8FEF8093EF038B
:1049E0008091EF038E3F09F4DDC0D4C00E946716AA
:1049F000882309F4D7C080915504882321F48FEFD0
:104A00008093EF03C7C080EF93E060E070E040E088
:104A100050E00E949C069B01AC018091EF03992716
:104A200087FD9095A92FB92FFC013197E930F10549
:104A300008F08CC0E753FF4F0C945E2FDA01C901D8
:104A40008154914EAD49B8418F57904FAA4FB24013
:104A500008F07CC02093C3033093C4034093C50384
:104A60005093C6039AC02093C7033093C803409362
:104A7000C9035093CA0381E0809356048EC0283046
:104A800031054105510508F061C02093CB0385C075
:104A9000DA01C9010197A109B1090A97A105B10578
:104AA00008F054C02093CC0378C080EF93E06DE30E
:104AB00071E00E94B80710E00EC0183130F4E12F09
:104AC000F0E0E254FC4F87871F5F80E090E06DE3E9
:104AD00071E00E94B807009759F00E949A0700976A
:104AE00061F706C0E12FF0E0E254FC4F17861F5F2C
:104AF0001831C0F352C0253031054105510530F55C
:104B00002093E5034AC0DA01C9010197A109B1095F
:104B10000697A105B105D0F48091E603887F822B2A
:104B20008093E6033AC0DA01C9010197A109B109EE
:104B30008050924CA140B04048F42093BF03309382
:104B4000C0034093C1035093C20327C085E296E09F
:104B500068EA71E00E946C2C13C08091C7039091A9
:104B6000C803A091C903B091CA030196A11DB11D4C
:104B70008093C7039093C803A093C903B093CA035B
:104B80000E945D168FEF8093EF0385E296E06AE066
:104B90000E940A2B0E94A41D05C080915604882300
:104BA000E1F2EECF1F9108958FEF8093EF03109203
:104BB00056040E94A41D0CC085E296E00E94B12D0F
:104BC000892B31F085E296E00E94EB2D0E94FF23B5
:104BD0008091EF038E3F81F76AE070E080E090E023
:104BE0000E94652904C085E296E00E94EB2D85E2D3
:104BF00096E00E94B12D892BB1F70895AAE2B0E0AA
:104C0000E4E0F6E20C942C2F0E9431297B018C0108
:104C100081E00E94640B04C085E296E00E94EB2DC7
:104C200085E296E00E94B12D892BB1F7439829982F
:104C3000DD24D394E2E67E2E72E0872E912C8C0E3A
:104C40009D1E5E010894A11CB11C63E0C62E0E944B
:104C5000312920E030E06E197F09800B910B693C0F
:104C600071058105910510F021E030E08D2D90E077
:104C700028233923232BB9F10E9431297B018C0190
:104C800085B1846285B980ED97E00E945E117982DA
:104C9000D401EEEBF3E089E201900D928150E1F74F
:104CA000C5016AE20E94720F85B18B7D85B980E0F3
:104CB00090E00E945E11C09298030E94430C62E350
:104CC00070E080E090E00E94652980919803843034
:104CD00051F4C09298038FE70E945A0A0E946E0A0C
:104CE000823409F4DD2487E00E94632A892B79F558
:104CF000DD24D3942CC0439A299A85B1846285B966
:104D000085E296E00E94EB2D8D30910569F08E30A2
:104D100091051CF40A97B1F407C08332910569F03C
:104D20008234910579F40CC085E296E064EA71E082
:104D30000E94F62A0E94D42505C00E94371E02C098
:104D40000E9452234398299885B18B7D85B985E2CD
:104D500096E00E94B12D892B09F479CFCCCF8F92A8
:104D60009F92AF92BF92CF92DF92EF92FF920F93FA
:104D70001F9387E00E94632A892B09F083C068ECA7
:104D800070E080E090E00E94652980E090E00E9461
:104D90005E110E9431295B016C01F0ECEF2EF2E113
:104DA000FF2E012D112DE60EF71E081F191F06C03C
:104DB00087E00E94632A892B09F062C00E94312992
:104DC0006E157F058007910798F387E00E94632A9C
:104DD000892B09F055C080ED97E00E945E110E947A
:104DE00031297B018C0199249394882488E496E2EC
:104DF000A0E0B0E0A80EB91ECA1EDB1E29C0AE148A
:104E0000BF04C006D10638F480ED97E00E945E1121
:104E1000882483941DC00E9431296E197F09800B5C
:104E2000910B693C71058105910590F00E94312933
:104E30007B018C0180E0992009F481E0982E882381
:104E400019F480E090E002C080ED97E00E945E11CE
:104E500087E00E94632A892B91F280E090E00E9413
:104E60005E11882049F0809199038F5F83700E94C2
:104E70004D160E94281606C00E9463230E941F162A
:104E80000E94FE251F910F91FF90EF90DF90CF9031
:104E9000BF90AF909F908F90089580E067EF77E08C
:104EA00042E050E00E946C280895EF92FF920F9329
:104EB0001F9380E00E9413080E94491181E161E084
:104EC0000E94C4298DE061E00E94C42989E061E06C
:104ED0000E94C4298AE061E00E94C42987E060E062
:104EE0000E94C42988E060E00E94C42988E061E053
:104EF0000E94302A0E943E1485E296E040E052EC87
:104F000061E070E00E942A2D0E9440160E9428163F
:104F10000E94080D8FEF8093AC040E944D27789477
:104F20000E9431297B018C018091AC048F3F09F0F4
:104F3000C8C00E9431296E197F09800B910B605DFA
:104F400077408040904008F0BCC0EECF85E296E00C
:104F50000E94EB2D85E296E00E94B12D892BB1F7DE
:104F600085E296E062E472E00E94692C82E693E0BA
:104F70000E94D01985E296E069E572E00E94692CF2
:104F800085E296E063E070E04AE050E00E94552C34
:104F900062E370E080E090E00E94652985E296E09F
:104FA0000E94B12D04970CF185E296E00E94EB2D52
:104FB00082349105D1F485E296E00E94EB2D8E3487
:104FC000910599F485E296E00E94EB2D84349105D9
:104FD00061F485E296E00E94EB2D819731F480E048
:104FE00090E00E945E110E94FE254091BF03509107
:104FF000C0036091C1037091C203DB01CA01019734
:10500000A109B1090497A105B10568F44093AD0465
:10501000433029F040E052EC61E070E004C040EA27
:1050200056E861E070E085E296E00E942A2D0E9439
:10503000AF264398299880E090E00E945E110E947C
:10504000080D80E00E94640B809192040E948F0AF8
:105050000E94430C10921705109218051092190522
:1050600010E015C062E370E080E090E00E946529E6
:1050700080ED97E00E945E1162E370E080E090E0D6
:105080000E94652980E090E00E945E111F5F809180
:105090009903811738F78091E60390E084FF09C0F7
:1050A00020E088719070489709F421E0822F0E94D7
:1050B00055148FE00E9413081F910F91FF90EF90FD
:1050C000089580ED97E00E945E1187E061E00E9404
:1050D000302A439A299A3ECF823000F5E82FF0E03B
:1050E000EE0FFF1FE057FA4F71836083882319F09A
:1050F0008130A1F408C0809169008C7F842B80935B
:105100006900E89A089580916900440F551F440F83
:10511000551F837F842B80936900E99A08951F921D
:105120000F920FB60F9211242F933F934F935F93DB
:105130006F937F938F939F93AF93BF93EF93FF935F
:105140008091900590919105892B29F0E09190052F
:10515000F09191050995FF91EF91BF91AF919F91CA
:105160008F917F916F915F914F913F912F910F9010
:105170000FBE0F901F9018951F920F920FB60F92AF
:1051800011242F933F934F935F936F937F938F934C
:105190009F93AF93BF93EF93FF938091920590916C
:1051A0009305892B29F0E0919205F09193050995DB
:1051B000FF91EF91BF91AF919F918F917F916F91EF
:1051C0005F914F913F912F910F900FBE0F901F90C5
:1051D00018951F920F920FB60F9211242F933F93A1
:1051E0008F939F93AF93BF9380919805909199056A
:1051F000A0919A05B0919B0530919C050196A11D47
:10520000B11D232F2D5F2D3720F02D570196A11DA5
:10521000B11D20939C058093980590939905A093C8
:105220009A05B0939B058091940590919505A09166
:105230009605B09197050196A11DB11D8093940527
:1052400090939505A0939605B0939705BF91AF9164
:105250009F918F913F912F910F900FBE0F901F90B4
:1052600018958FB7F8942091980530919905409141
:105270009A0550919B058FBFB901CA0108959FB748
:10528000F8942091940530919505409196055091A0
:10529000970586B5A89B06C08F3F21F02F5F3F4F33
:1052A0004F4F5F4F9FBF542F432F322F2227280F7E
:1052B000311D411D511D82E0220F331F441F551F18
:1052C0008A95D1F7B901CA010895EF92FF920F9321
:1052D0001F93CF93DF937B018C010E943F29EB0149
:1052E0000EC00E943F296C1B7D0B685E7340C8F3A3
:1052F0000894E108F10801091109C851DC4FE114D3
:10530000F1040105110569F7CDB7DEB7E6E00C94AD
:105310004F2F789484B5826084BD84B5816084BD4C
:1053200085B5826085BD85B5816085BDEEE6F0E01E
:10533000808181608083E1E8F0E01082808182607A
:105340008083808181608083E0E8F0E080818160FB
:105350008083E1EBF0E0808184608083E0EBF0E02B
:10536000808181608083EAE7F0E0808184608083CF
:105370008081826080838081816080838081806879
:1053800080831092C1000895CF93DF93482F50E09F
:10539000CA018850944FFC0134914C51544FFA018A
:1053A0008491882369F190E0880F991FFC01EA53EA
:1053B000F44FA591B491FC01E053F44FC591D49101
:1053C000662351F42FB7F8948C91932F90958923ED
:1053D0008C93888189230BC0623061F42FB7F894D5
:1053E0008C91932F909589238C938881832B88832C
:1053F0002FBF06C09FB7F8948C91832B8C939FBFCF
:10540000DF91CF910895833071F0843028F481309A
:10541000A1F0823021F514C08630B1F08730D1F090
:105420008430E9F404C0809180008F7703C08091BC
:1054300080008F7D80938000089584B58F7702C0AF
:1054400084B58F7D84BD08958091B0008F7780935F
:10545000B00008958091B0008F7D8093B0000895D2
:10546000FF920F931F93F62E482F50E0CA01845FDE
:10547000934FFC012491CA018850944FFC01149170
:105480004C51544FFA0104910023C9F0222319F022
:10549000822F0E94032AE02FF0E0EE0FFF1FE0535F
:1054A000F44FA591B4919FB7F894FF2021F48C910B
:1054B0001095812302C08C91812B8C939FBF1F91EB
:1054C0000F91FF9008950F931F93482F50E0CA014A
:1054D000845F934FFC012491CA018850944FFC01D2
:1054E00004914C51544FFA011491112319F420E006
:1054F00030E015C0222319F0822F0E94032A812F49
:1055000090E0880F991F8652944FFC01A591B491A9
:105510008C9120E030E0802311F021E030E0C901DF
:105520001F910F910895A0E0B0E0E9E9FAE20C9430
:10553000312F7C016B018A01C0E0D0E00FC0D601A1
:105540006D916D01D701ED91FC910190F081E02DFD
:10555000C7010995C80FD91F015010400115110549
:1055600071F7CE01CDB7DEB7E8E00C944D2FEF9286
:10557000FF920F931F93CF93DF937C018B01C0E0C9
:10558000D0E0F8010F5F1F4F6491662359F0D701F7
:10559000ED91FC910190F081E02DC7010995C80FB4
:1055A000D91FEFCFCE01CDB7DEB7E6E00C944F2F79
:1055B000DC01ED91FC910190F081E02D09950895B9
:1055C000EF92FF920F931F938C016DE00E94D82AF7
:1055D0007C01C8016AE00E94D82A9C012E0D3F1D63
:1055E000C9011F910F91FF90EF900895EF92FF92E4
:1055F0000F931F937C010E94B72A8C01C7010E9460
:10560000E02A9C01200F311FC9011F910F91FF90CB
:10561000EF900895EF92FF920F931F937C010E94E9
:10562000D82A8C01C7010E94E02A9C01200F311F5B
:10563000C9011F910F91FF90EF900895CF93DF93D1
:10564000EC016115710519F420E030E00FC0DB01B9
:105650000D900020E9F71197A61BB70BE881F9819F
:105660000280F381E02DAD0109959C01C901DF9114
:10567000CF9108954F925F927F928F929F92AF92B7
:10568000BF92CF92DF92EF92FF920F931F93DF931F
:10569000CF93CDB7DEB7A1970FB6F894DEBF0FBE9C
:1056A000CDBF2C01742ECB01223008F42AE019A2C0
:1056B00031E2C32ED12CCC0EDD1E822E9924AA24D9
:1056C000BB24672D752FA50194010E94EA2E790154
:1056D0008A01C801B701A50194010E94B82E472D87
:1056E000461B0894C108D1084A3010F4405D01C03F
:1056F000495CF6014083E114F1040105110521F034
:105700007E2C5F2DC801DDCFC201B6010E941E2B89
:10571000A1960FB6F894DEBF0FBECDBFCF91DF913B
:105720001F910F91FF90EF90DF90CF90BF90AF90BF
:105730009F908F907F905F904F900895DC0121158E
:10574000310541F4ED91FC910190F081E02D642F41
:10575000099508950E943A2B0895EF92FF920F93B6
:105760001F937C010E949E2B8C01C7010E94E02A9E
:105770009C01200F311FC9011F910F91FF90EF90E5
:105780000895EF92FF920F931F939A017B0100E01F
:1057900010E0B801A7010E949E2B1F910F91FF906E
:1057A000EF900895EF92FF920F931F937C010E9458
:1057B000C12B8C01C7010E94E02A9C01200F311FE0
:1057C000C9011F910F91FF90EF900895EF92FF9202
:1057D0000F931F939A01E62EFF2400E010E0B8011A
:1057E000A7010E949E2B1F910F91FF90EF900895AB
:1057F000EF92FF920F931F937C010E94E62B8C0186
:10580000C7010E94E02A9C01200F311FC9011F918E
:105810000F91FF90EF900895A0E0B0E0E2E1FCE28C
:105820000C94312FEC016A017B012115310541F403
:10583000E881F9810190F081E02D642F09951BC06A
:105840002A303105B1F477FF13C06DE20E94D82AE7
:105850008C0144275527BA014C195D096E097F094F
:10586000CE012AE00E943A2B9C01200F311F04C078
:105870002AE00E943A2B9C01C901CDB7DEB7E8E0CF
:105880000C944D2FEF92FF920F931F937B019A017F
:105890000027F7FC0095102FB801A7010E940C2CDF
:1058A0001F910F91FF90EF900895EF92FF920F9349
:1058B0001F937C010E94422C8C01C7010E94E02AA8
:1058C0009C01200F311FC9011F910F91FF90EF9094
:1058D00008950E941E2B0895EF92FF920F931F933D
:1058E0007C010E94692C8C01C7010E94E02A9C0166
:1058F000200F311FC9011F910F91FF90EF90089564
:1059000008951F920F920FB60F9211242F933F9379
:105910004F938F939F93EF93FF938091C00082FDED
:105920001DC04091C6002091DD053091DE052F5F3E
:105930003F4F2F7330708091DF059091E00528175D
:10594000390771F0E091DD05F091DE05E356FA4F7D
:1059500040833093DE052093DD0502C08091C600B0
:10596000FF91EF919F918F914F913F912F910F90C8
:105970000FBE0F901F9018951F920F920FB60F92A7
:1059800011242F933F938F939F93EF93FF93209135
:105990002106309122068091230690912406281733
:1059A000390731F48091C1008F7D8093C10014C00C
:1059B000E0912306F0912406EF51FA4F2081809167
:1059C00023069091240601968F739070909324067D
:1059D000809323062093C600FF91EF919F918F91B2
:1059E0003F912F910F900FBE0F901F901895A0E040
:1059F000B0E0EDEFFCE20C942D2FFC01138212823B
:105A000088EE93E0A0E0B0E084839583A683B7831B
:105A10008AE893E0918380837587648757874687F8
:105A2000318B208B138B028BF58AE48AD78AC68A46
:105A3000B18EA08E938E828E8F85848F8889858F7C
:105A40008989868F8A89878F8B8980A32096ECE04D
:105A50000C94492FAF92BF92DF92EF92FF920F9377
:105A60001F93CF93DF93EC017A018B01DD2440304B
:105A700081EE580780E0680780E0780711F0DD24A8
:105A8000D39491E0A92EB12CEC89FD89DD2069F039
:105A9000C50108A002C0880F991F0A94E2F780830D
:105AA00060E079E08DE390E005C0108260E874E882
:105AB0008EE190E0A80197010E94EA2E215030402B
:105AC00040405040569547953795279580E12030C6
:105AD000380720F0DD2011F0DD24D6CFE889F989E0
:105AE0003083EA89FB89208319A2EE89FF894081EE
:105AF00021E030E0C9010C8C02C0880F991F0A9484
:105B0000E2F7482B4083EE89FF894081C9010D8C63
:105B100002C0880F991F0A94E2F7482B4083EE8950
:105B2000FF894081C9010E8C02C0880F991F0A9419
:105B3000E2F7482B4083EE89FF8980810F8C02C0F9
:105B4000220F331F0A94E2F7209528232083DF9148
:105B5000CF911F910F91FF90EF90DF90BF90AF908A
:105B60000895DC011C96ED91FC911D97E05CFF4FC0
:105B70002191319180819181281B390B2F733070D5
:105B8000C901089585E296E00E94B12D892B11F09C
:105B90000E94802C0895DC011C96ED91FC911D97CC
:105BA000E05CFF4F20813181E054F040DF01AE5BCB
:105BB000BF4F8D919C9111972817390719F42FEF3A
:105BC0003FEF07C08D919C91E80FF91F8081282F2E
:105BD00030E0C9010895DC011C96ED91FC911D9700
:105BE000E05CFF4F20813181E054F040DF01AE5B8B
:105BF000BF4F8D919C9111972817390719F42FEFFA
:105C00003FEF10C08D919C911197E80FF91F2081F3
:105C10008D919C91119701968F73907011969C9322
:105C20008E9330E0C9010895DC0191968C91919793
:105C3000882339F05496ED91FC915597808186FF29
:105C4000F9CF91961C920895CF93DF93EC01EE85E6
:105C5000FF85E05CFF4F20813181E054F0402F5FF1
:105C60003F4F2F733070DF01AE5BBF4F8D919C9122
:105C7000119728173907D1F3E05CFF4F808191819C
:105C8000E054F040E80FF91F6083EE85FF85E05C8B
:105C9000FF4F31832083EE89FF89208181E090E0EE
:105CA0000F8C02C0880F991F0A94E2F7282B2083DB
:105CB00081E089A3EC89FD8980818064808381E013
:105CC00090E0DF91CF9108958F929F92AF92BF9213
:105CD000CF92DF92EF92FF920F931F9300D000D0EC
:105CE0000F92EDB7FEB7319684E0ADB7BEB711960F
:105CF0008C9383E0818387E0828385E0838381E0E6
:105D0000848385E296E06DE975E041EE55E025EC8F
:105D100030E004EC10E0B0ECEB2EF12CA1ECCA2E3C
:105D2000D12CF2ECAF2EB12CE6EC8E2E912C0E94F1
:105D3000F72C0F900F900F900F900F901F910F91D5
:105D4000FF90EF90DF90CF90BF90AF909F908F909B
:105D50000895CF93DF930E9489290E945527C2ECB2
:105D6000DDE20E9497112097E1F30E94C22DF9CF46
:105D7000629FD001739FF001829FE00DF11D649F2F
:105D8000E00DF11D929FF00D839FF00D749FF00DBB
:105D9000659FF00D9927729FB00DE11DF91F639F5C
:105DA000B00DE11DF91FBD01CF011124089597FB2E
:105DB000092E07260AD077FD04D086D006D0002011
:105DC0001AF4709561957F4F0895F6F79095819537
:105DD0009F4F0895A1E21A2EAA1BBB1BFD010DC007
:105DE000AA1FBB1FEE1FFF1FA217B307E407F5078B
:105DF00020F0A21BB30BE40BF50B661F771F881F67
:105E0000991F1A9469F760957095809590959B01FC
:105E1000AC01BD01CF01089597FB092E05260ED0D8
:105E200057FD04D0D7DF0AD0001C38F450954095B8
:105E3000309521953F4F4F4F5F4F0895F6F790955E
:105E40008095709561957F4F8F4F9F4F08952F924A
:105E50003F924F925F926F927F928F929F92AF92FA
:105E6000BF92CF92DF92EF92FF920F931F93CF9347
:105E7000DF93CDB7DEB7CA1BDB0B0FB6F894DEBFDE
:105E80000FBECDBF09942A88398848885F846E8404
:105E90007D848C849B84AA84B984C884DF80EE804E
:105EA000FD800C811B81AA81B981CE0FD11D0FB657
:105EB000F894DEBF0FBECDBFED010895EE0FFF1FBA
:105EC0000590F491E02D0994AA1BBB1B51E107C07A
:105ED000AA1FBB1FA617B70710F0A61BB70B881F7A
:105EE000991F5A95A9F780959095BC01CD01089509
:105EF000911106C0803219F089508550D0F708956D
:0A5F0000992788270895F894FFCF31
:105F0A004E6F005965730054582074696D656F753A
:105F1A007421006D6F64756C65206C6F636B6564CA
:105F2A003F00486F70206368616E6E656C200020C8
:105F3A0040200053004E2F4100386368002C002C8B
:105F4A00205B005D20280029004E4F5420454E4119
:105F5A00424C45440053656E64696E6720736574EC
:105F6A0074696E677320746F2052580A0052657301
:105F7A00657474696E672073657474696E677320DB
:105F8A006F6E2052580A0041626F72746564206510
:105F9A00646974730A00696E76616C69642073655A
:105FAA006C656374696F6E000D0A496E76616C697F
:105FBA006420696E707574202D2064697363617240
:105FCA006465642107007363616E6E6572206D6F8C
:105FDA0064650053657474696E67732073617665CE
:105FEA006420746F20454550524F4D0A0052657621
:105FFA0065727465642073657474696E677320666C
:10600A00726F6D20454550524F4D0A004C6F6164C6
:10601A00656420666163746F727920646566617570
:10602A006C74730A004B657920616E642063686141
:10603A006E6E656C732072616E646F6D697A6564E9
:10604A000A004F70656E4C52536E67205458207385
:10605A0074617274696E672000206F6E2048572041
:10606A000050504D0052535349005344410053438A
:10607A004C00525844005458440041494E004C4286
:10608A004545500053504B54524D0053425553000E
:10609A0053554D44004C4C494E440000342B3400B7
:1060AA003800382B340031320031322B340031368B
:1060BA000001000000C01200001A400AA1204EA5EB
:1060CA00001B1E27522C23308025000005400AA100
:1060DA00204EA50020244EA52C2330004B0000069C
:1060EA00400AD0009D49007B289D492C233000E1BD
:1060FA00000005400A4501D7DC03B81E0EBF002385
:10610A002E48E801008A400A6001555502AD1E205A
:10611A00000023C88025000005400AA1204EA500E2
:10612A0020244EA52C2330000200020002000200A7
:10613A000200020002000200020002000200020045
:10614A0002000200020002FF610265026A026E0298
:10615A00720276027A027E0284028B029002950211
:10616A009B029B029B029B0235019C02A002A20297
:10617A00A602A902AE02350100070B0C1011150088
:10618A00160A1322312900000000242E932AB12D69
:06619A00EB2DCB2D142EAD
:00000001FF
